
UART Transmission Reception.elf:     file format elf32-avr

Sections:
Idx Name          Size      VMA       LMA       File off  Algn
  0 .text         0000006c  00000000  00000000  00000054  2**1
                  CONTENTS, ALLOC, LOAD, READONLY, CODE
  1 .data         00000000  00800060  00800060  000000f4  2**0
                  ALLOC, LOAD, DATA
  2 .comment      0000002f  00000000  00000000  000000f4  2**0
                  CONTENTS, READONLY
  3 .debug_aranges 00000030  00000000  00000000  00000123  2**0
                  CONTENTS, READONLY, DEBUGGING
  4 .debug_info   000007d0  00000000  00000000  00000153  2**0
                  CONTENTS, READONLY, DEBUGGING
  5 .debug_abbrev 00000554  00000000  00000000  00000923  2**0
                  CONTENTS, READONLY, DEBUGGING
  6 .debug_line   0000020f  00000000  00000000  00000e77  2**0
                  CONTENTS, READONLY, DEBUGGING
  7 .debug_frame  00000044  00000000  00000000  00001088  2**2
                  CONTENTS, READONLY, DEBUGGING
  8 .debug_str    00000196  00000000  00000000  000010cc  2**0
                  CONTENTS, READONLY, DEBUGGING
  9 .debug_loc    00000040  00000000  00000000  00001262  2**0
                  CONTENTS, READONLY, DEBUGGING
 10 .debug_ranges 00000020  00000000  00000000  000012a2  2**0
                  CONTENTS, READONLY, DEBUGGING
 11 .text         00000004  0000009c  0000009c  000000f0  2**1
                  CONTENTS, ALLOC, LOAD, READONLY, CODE
 12 .note.gnu.avr.deviceinfo 0000003c  00000000  00000000  000012c4  2**2
                  CONTENTS, READONLY, DEBUGGING
 13 .text.transmit 0000000c  00000088  00000088  000000dc  2**1
                  CONTENTS, ALLOC, LOAD, READONLY, CODE
 14 .text.receive 00000008  00000094  00000094  000000e8  2**1
                  CONTENTS, ALLOC, LOAD, READONLY, CODE
 15 .text.main    0000001c  0000006c  0000006c  000000c0  2**1
                  CONTENTS, ALLOC, LOAD, READONLY, CODE

Disassembly of section .text:

00000000 <__vectors>:
   0:	0c 94 2a 00 	jmp	0x54	; 0x54 <__ctors_end>
   4:	0c 94 4e 00 	jmp	0x9c	; 0x9c <__bad_interrupt>
   8:	0c 94 4e 00 	jmp	0x9c	; 0x9c <__bad_interrupt>
   c:	0c 94 4e 00 	jmp	0x9c	; 0x9c <__bad_interrupt>
  10:	0c 94 4e 00 	jmp	0x9c	; 0x9c <__bad_interrupt>
  14:	0c 94 4e 00 	jmp	0x9c	; 0x9c <__bad_interrupt>
  18:	0c 94 4e 00 	jmp	0x9c	; 0x9c <__bad_interrupt>
  1c:	0c 94 4e 00 	jmp	0x9c	; 0x9c <__bad_interrupt>
  20:	0c 94 4e 00 	jmp	0x9c	; 0x9c <__bad_interrupt>
  24:	0c 94 4e 00 	jmp	0x9c	; 0x9c <__bad_interrupt>
  28:	0c 94 4e 00 	jmp	0x9c	; 0x9c <__bad_interrupt>
  2c:	0c 94 4e 00 	jmp	0x9c	; 0x9c <__bad_interrupt>
  30:	0c 94 4e 00 	jmp	0x9c	; 0x9c <__bad_interrupt>
  34:	0c 94 4e 00 	jmp	0x9c	; 0x9c <__bad_interrupt>
  38:	0c 94 4e 00 	jmp	0x9c	; 0x9c <__bad_interrupt>
  3c:	0c 94 4e 00 	jmp	0x9c	; 0x9c <__bad_interrupt>
  40:	0c 94 4e 00 	jmp	0x9c	; 0x9c <__bad_interrupt>
  44:	0c 94 4e 00 	jmp	0x9c	; 0x9c <__bad_interrupt>
  48:	0c 94 4e 00 	jmp	0x9c	; 0x9c <__bad_interrupt>
  4c:	0c 94 4e 00 	jmp	0x9c	; 0x9c <__bad_interrupt>
  50:	0c 94 4e 00 	jmp	0x9c	; 0x9c <__bad_interrupt>

00000054 <__ctors_end>:
  54:	11 24       	eor	r1, r1
  56:	1f be       	out	0x3f, r1	; 63
  58:	cf e5       	ldi	r28, 0x5F	; 95
  5a:	d8 e0       	ldi	r29, 0x08	; 8
  5c:	de bf       	out	0x3e, r29	; 62
  5e:	cd bf       	out	0x3d, r28	; 61
  60:	0e 94 36 00 	call	0x6c	; 0x6c <_etext>
  64:	0c 94 34 00 	jmp	0x68	; 0x68 <_exit>

00000068 <_exit>:
  68:	f8 94       	cli

0000006a <__stop_program>:
  6a:	ff cf       	rjmp	.-2      	; 0x6a <__stop_program>

Disassembly of section .text:

0000009c <__bad_interrupt>:
  9c:	0c 94 00 00 	jmp	0	; 0x0 <__TEXT_REGION_ORIGIN__>

Disassembly of section .text.transmit:

00000088 <transmit>:
	}	
}
	
	
void transmit(char a){
	UDR=a;
  88:	8c b9       	out	0x0c, r24	; 12
	while((UCSRA&0x40)==0);
  8a:	5e 9b       	sbis	0x0b, 6	; 11
  8c:	fe cf       	rjmp	.-4      	; 0x8a <transmit+0x2>
	UCSRA=0x40;
  8e:	80 e4       	ldi	r24, 0x40	; 64
  90:	8b b9       	out	0x0b, r24	; 11
  92:	08 95       	ret

Disassembly of section .text.receive:

00000094 <receive>:
}

char receive(){
	while((UCSRA&0x80)==0);
  94:	5f 9b       	sbis	0x0b, 7	; 11
  96:	fe cf       	rjmp	.-4      	; 0x94 <receive>
	return(UDR);
  98:	8c b1       	in	r24, 0x0c	; 12
}	
  9a:	08 95       	ret

Disassembly of section .text.main:

0000006c <main>:
void transmit(char);
char receive();

int main()
{	
	DDRD=0X02;
  6c:	82 e0       	ldi	r24, 0x02	; 2
  6e:	81 bb       	out	0x11, r24	; 17
	char a;
	UBRRL=0x33;
  70:	83 e3       	ldi	r24, 0x33	; 51
  72:	89 b9       	out	0x09, r24	; 9
	UBRRH=0x00;
  74:	10 bc       	out	0x20, r1	; 32
	UCSRB=0x18;
  76:	88 e1       	ldi	r24, 0x18	; 24
  78:	8a b9       	out	0x0a, r24	; 10
	UCSRC=0x86;
  7a:	86 e8       	ldi	r24, 0x86	; 134
  7c:	80 bd       	out	0x20, r24	; 32
	int i;
	
	while(1){
		a=receive();
  7e:	0e 94 4a 00 	call	0x94	; 0x94 <receive>
		transmit(a);	
  82:	0e 94 44 00 	call	0x88	; 0x88 <transmit>
  86:	fb cf       	rjmp	.-10     	; 0x7e <main+0x12>
